:020000040000FA
:10000000D9043700B40900002E0C0000420C000097
:10001000560C00006E0C0000880C00009E0C0000C6
:10002000B80C0000CC0C0000DE0C0000DE0C000060
:10003000DE0C0000DE0C0000DE0C0000DE0C000018
:10004000DE0C0000020E0000DE0C0000DE0C0000E2
:10005000DE0C0000C60D0000DE0C0000DE0C00000F
:10006000DE0C0000DE0C0000DE0C0000DE0C0000E8
:10007000DE0C0000DE0C0000DE0C0000DE0C0000D8
:10008000DE0C0000DE0C0000DE0C0000DE0C0000C8
:10009000DE0C0000DE0C0000DE0C0000DE0C0000B8
:1000A000DE0C0000DE0C0000DE0C0000DE0C0000A8
:1000B000DE0C0000DE0C0000DE0C0000DE0C000098
:1000C000DE0C0000DE0C0000DE0C0000DE0C000088
:1000D000DE0C0000DE0C0000DE0C0000DE0C000078
:1000E000DE0C0000DE0C0000DE0C0000DE0C000068
:1000F000DE0C0000DE0C0000DE0C0000DE0C000058
:10010000DE0C0000DE0C0000DE0C0000DE0C000047
:10011000DE0C0000DE0C0000DE0C0000DE0C000037
:10012000DE0C0000DE0C0000DE0C0000DE0C000027
:10013000DE0C0000DE0C0000DE0C0000DE0C000017
:10014000DE0C0000DE0C0000DE0C0000DE0C000007
:10015000DE0C0000DE0C0000DE0C0000DE0C0000F7
:10016000DE0C0000DE0C0000DE0C0000DE0C0000E7
:10017000DE0C0000DE0C0000DE0C0000DE0C0000D7
:10018000DE0C0000DE0C0000DE0C0000DE0C0000C7
:10019000DE0C0000DE0C0000DE0C0000DE0C0000B7
:1001A000DE0C0000DE0C0000DE0C0000DE0C0000A7
:1001B000DE0C0000DE0C0000DE0C0000DE0C000097
:1001C000DE0C0000DE0C0000DE0C0000DE0C000087
:1001D000DE0C0000DE0C0000DE0C0000DE0C000077
:1001E000DE0C0000DE0C0000DE0C0000DE0C000067
:1001F000DE0C0000DE0C0000DE0C0000DE0C000057
:100200000027000002270000042700000627000046
:10021000082700000A2700000C2700000E27000016
:1002200010270000122700001427000016270000E6
:10023000182700001A2700001C2700001E270000B6
:100240002027000022270000242700002627000086
:10025000282700002A2700002C2700002E27000056
:100260003027000032270000342700003627000026
:10027000382700003A2700003C2700003E270000F6
:1002800040270000422700004427000046270000C6
:10029000482700004A2700004C2700004E27000096
:1002A0005027000052270000542700005627000066
:1002B000582700005A2700005C2700005E27000036
:1002C0006027000062270000642700006627000006
:1002D000682700006A2700006C2700006E270000D6
:1002E00070270000722700007427000076270000A6
:1002F000782700007A2700007C2700007E27000076
:100300008027000082270000842700008627000045
:10031000882700008A2700008C2700008E27000015
:1003200090270000922700009427000096270000E5
:10033000982700009A2700009C2700009E270000B5
:10034000A0270000A2270000A4270000A627000085
:10035000A8270000AA270000AC270000AE27000055
:10036000B0270000B2270000B4270000B627000025
:10037000B8270000BA270000BC270000BE270000F5
:10038000C0270000C2270000C4270000C6270000C5
:10039000C8270000CA270000CC270000CE27000095
:1003A000D0270000D2270000D4270000D627000065
:1003B000D8270000DA270000DC270000DE27000035
:1003C000E0270000E2270000E4270000E627000005
:1003D000E8270000EA270000EC270000EE270000D5
:1003E000F0270000F2270000F4270000F6270000A5
:1003F000F8270000FA270000FC270000FE27000075
:1004000000C0B300ECEAB70060EDB70061EDB700E3
:100410006AEDB70066EDB700CCEAB700FAEAB700BC
:1004200010002000F9EAB70020002000F8EAB70029
:1004300030002000F7EAB70040002000F5EAB700DE
:1004400080002000F4EAB700F0CFB300F3EAB70071
:10045000F00F20006BEDB700800F2000F2EAB7002C
:1004600010002000F1EAB700B0002000F0EAB70069
:10047000000C2000D3EAB70080002000DDEAB700BE
:10048000B0002000DCEAB70000002000E4EAB7007A
:1004900000002000E5EAB70000002000E0EAB70015
:1004A00000002000E1EAB700C0FE2000EAAAB70081
:1004B0002882BF000020EC002062AF00020037005D
:1004C0004100DD00010037004200DD0064AAB700F2
:1004D0000020EF006BCDBF00BA0AB400640ABC0074
:1004E0000680BF0003003A000480BF000CA1B700E3
:1004F000010037000CA1EF00C482A900803E20005B
:100500002AAAB7002C2AEC0061CDBF0002003A00F5
:10051000C482A90001003700CDE2A90000E020005C
:1005200014A0B700CB6AEF008C6AEF00E96AEF0015
:1005300066050700ECCABF0088EAB70000CCB3002C
:10054000EC4AB600F8FF3200CBEAEF00F0C1B3008E
:10055000884AB600D2EAB70000CCB300884AB60099
:10056000D3EAB70000CCB300D34AB50004003A0088
:10057000F0CFB300884AB50001003A00E7FF37002A
:1005800000C8B300D34AB50016003A00F0C3B30068
:10059000884AB600D1EAB700E9EAEF00D1CABF0045
:1005A0004200A90000C0D60000C0D60000C0D6009E
:1005B00000C0D60017E0B70000C0D700F24AB6006E
:1005C00016E0B70017C0BF00F14AB600F04AB40009
:1005D00017E0B700C4E9EF003B40780088EAB700B5
:1005E0000000370088CABF00005D780000CCB3006F
:1005F000884AB600D3EAB700F0C3B300884AB60011
:10060000D1EAB70080C0B300884AB600CEEAB7008E
:1006100040C0B300884AB600EEEAB70030C0B3006D
:10062000884AB600EDEAB70000C2B300884AB600B7
:10063000EFEAB70000CCB300D34AB5000A003A0095
:1006400000C2B300EF4AB50007003A0000C0B30093
:10065000E94AB500030032000B409000005D7800CD
:10066000010037004505070000C4B300D34AB500B8
:1006700065003A0040C0B300EE4AB5000A003A00F7
:1006800000C0B300E94AB500050032003B407800E5
:10069000005D78003B407800005D78000200370084
:1006A000360507003505070000C2B300EF4AB50064
:1006B00055003A0000C0B300ED4AB5000A003A0008
:1006C00000C1B300884AB6000600320000C0B30083
:1006D000E94AB500020032003B407800005D780036
:1006E000010037002505070010C0B300ED4AB50032
:1006F0000D003A0000C1B300884AB600080032007D
:1007000000C0B300E94AB500040032003B40780065
:10071000005D78003B407800005D78000200370003
:10072000160507001505070020C0B300ED4AB50007
:1007300013003A0000C1B300884AB6000C00320032
:1007400000C0B300E94AB500080032003B40780021
:10075000005D78003B407800005D78003B40780009
:10076000005D78003B407800005D780004003700B1
:10077000020507000105070000050700FF04070048
:1007800030C0B300ED4AB5001F003A0000C1B3000D
:10079000884AB6001400320000C0B300E94AB50030
:1007A000100032003B407800005D78003B4078004C
:1007B000005D78003B407800005D78003B407800A9
:1007C000005D78003B407800005D78003B40780099
:1007D000005D78003B407800005D78003B40780089
:1007E000005D780008003700E4040700E304070018
:1007F000E2040700E1040700E0040700DF0407004B
:10080000DE040700DD04070000C0B300E94AB500BC
:1008100002003A0000C0B30088EAB70000C0B3008D
:100820000045980000C0B300E94AB5000A00320054
:100830003B40780088EAB700005D780014C0BF0034
:10084000EA4AB50015C0BF00EBCAB500020031008E
:1008500000C1B300616DB70088CABF0063FF3A00F2
:10086000E96AEF0000C0B3000045980062CDBF0008
:10087000090032008CCABF0078040700ECCABF0030
:100880008C4AB5000400320010C0B300616DB7009F
:10089000636DEC0021FF3700CB6AEF0000E0200021
:1008A00014A0B7008B6AEF003A40780088EAB700DE
:1008B00000CCB300884AB600D3EAB70080C0B300CA
:1008C000884AB600CEEAB70040C0B300884AB600F6
:1008D000EEEAB70030C0B300884AB600EDEAB700D0
:1008E00000C2B300884AB600EFEAB70000CCB300FC
:1008F000D34AB500BF003A00F0C1B300884AB60041
:10090000D2EAB70000C2B300884AB600EFEAB700E7
:1009100016C0BF00E2EAB70017C0BF00E3EAB700A5
:1009200000C1B300D24AB5001100310000D620004A
:1009300016A0B70016C0BF00D24AB40016E0B70038
:1009400017C0BF00FACAB40017E0B70000C2B30076
:10095000EF4AB50003003A003A407800804598001D
:10096000020037000B4090007A0407009D0037001A
:1009700000C2B300EF4AB50042003A0070CFB300A6
:10098000884AB50002003A003A4078003C0037003F
:1009900080CFB300884AB50009003A0000C0B30018
:1009A0006A4DB50003003A003A407800E4EAB70027
:1009B000020037003A407800E0EAB7003000370024
:1009C00090CFB300884AB50009003A0000C0B300D8
:1009D0006A4DB50003003A003A407800E5EAB700F6
:1009E000020037003A407800E1EAB70024003700FF
:1009F000A0CFB300884AB50011003A0000C0B30090
:100A00006A4DB50007003A003A407800E44AB40065
:100A1000E4EAB700E5CABF00FACAB400E5EAB700E5
:100A2000060037003A407800E04AB400E0EAB70038
:100A3000E1CABF00FACAB400E1EAB700100037000B
:100A4000D0CFB300884AB50003003A003A4078009E
:100A5000CCEAB7000A003700E0CFB300884AB500FF
:100A600007003A003A407800ECEAB700A0C5B300AE
:100A7000EC4AB50001003A003B02370000003700A5
:100A80005800370000CDB300884AB50003003A0093
:100A900070C3B3002F0407005200370010CDB3001D
:100AA000884AB50003003A0090C4B3002904070047
:100AB0004C00370020CDB300884AB50003003A004F
:100AC00070C3B300230407004600370030CDB300E5
:100AD000884AB50003003A0070C3B3001D04070044
:100AE0004000370040CDB300884AB50003003A000B
:100AF000D0C0B300170407003A00370050CDB30050
:100B0000884AB50003003A00E7CABF001104070095
:100B10003400370060CDB300884AB50003003A00C6
:100B2000E6CABF000B0407002E00370070CDB300EB
:100B3000884AB50003003A0040C9BF000504070019
:100B400028003700A0CDB300884AB50003003A0062
:100B500000C0B300FF03070022003700C0CDB30080
:100B6000884AB50003003A0080C0B300F9030700CB
:100B70001C00370080CDB300884AB50008003A0059
:100B800000C0B3006A4DB50002003A00E4CABF00DD
:100B900001003700E0CABF00EE0307001100370074
:100BA00090CDB300884AB50008003A0000C0B300F9
:100BB0006A4DB50002003A00E5CABF0001003700E7
:100BC000E1CABF00E303070006003700F0CDB30021
:100BD000884AB50003003A00A0C5B300DD03070052
:100BE00000003700E2CABF0016E0B700E3CABF004A
:100BF00017E0B700F0C3B300884AB600D1EAB700E7
:100C000000C4B300D34AB500CD013A0040C0B300E0
:100C1000EE4AB5000C003A0000C0B3006A4DB500C2
:100C200005003A003A407800E4EAB7003A4078001C
:100C3000E5EAB700040037003A407800E0EAB70080
:100C40003A407800E1EAB70000C0B3006A4DB50051
:100C500005003A00E4CABF0016E0B700E5CABF00CD
:100C600017E0B70005003700E0CABF0016E0B70084
:100C7000E1CABF00F04AB40017E0B70020C0B300DB
:100C80006C4DB50002003A004200A9000600370092
:100C900000C0B3006A4DB50002003A004200A9004E
:100CA000010037004200A9000400390000DB2000E9
:100CB00016A0B70000C2B300616DB70010C0B3004A
:100CC0006C4DB50016003A003220EF004200F800EB
:100CD000000E20004200B70042A0B70000DB200059
:100CE0001AA0B70000802200E44AB40018A0B700A0
:100CF00080002000ACAAB7001880BF001040BA00E6
:100D0000804698001820EC001A20EC00AC2AED0078
:100D1000F9FF3A0000DB200016A0B7004200F900FE
:100D200020C0B3006C4DB50034003A0080002000B4
:100D3000DDEAB700B0002000DCEAB7004200A900FD
:100D4000DA8ABF000080D700D6AAB700D88ABF00D1
:100D50000080D7000000A900D4AAB700F0FF270048
:100D6000E40AB6004200A9000080D7000000A900F4
:100D7000D40AB400D4AAB70000C8B300E54AB6004C
:100D80001B003A0000DB200016A0B70000C2B30031
:100D9000EF4AB500150032001400F800D68ABF00F3
:100DA00032A0B700D48ABF0014A0B70000DB200037
:100DB0001AA0B7001480BF001000BA00801E78008F
:100DC0001480BF001080BA00801E780014A0EC00D0
:100DD0001480BF001000BA00801E78001480BF008D
:100DE0001080BA00801E78001400F900030037005C
:100DF00080AD2000E44AB40016A0B70000C2B300E2
:100E0000EF4AB500FA003A0000C0B300ED4AB50061
:100E100004003A003A407800805D7800F9CABF00CB
:100E2000F702070010C0B300ED4AB50007003A0012
:100E30000400FC003A407800805D78003A40780079
:100E4000805D7800F8CABF00ED02070020C0B30043
:100E5000ED4AB5000B003A000800FC003A4078006B
:100E6000805D78003A407800805D78003A407800F4
:100E7000805D78003A407800805D7800F5CABF0058
:100E8000DF02070030C0B300ED4AB50013003A009E
:100E90001000FC003A407800805D78003A4078000D
:100EA000805D78003A407800805D78003A407800B4
:100EB000805D78003A407800805D78003A407800A4
:100EC000805D78003A407800805D78003A40780094
:100ED000805D7800F4CABF00C902070010C0B300EB
:100EE0006C4DB50052003A003220EF004200F8008D
:100EF000000E20004200B70042A0B700E5CABF00C4
:100F000047003A0000C8B300E44AB60040003A0087
:100F10001400F8000080220014A0B7000004200094
:100F2000ACAAB7001480BF001000BA00000DBB00CF
:100F300000002000008DBB0014A0EC00AC2AED00E6
:100F4000F8FF3A003220EF002004240060A7B70029
:100F50000080220014A0B7001000BA00000DBB00F2
:100F600040A7A9004200F800000E20004200B70090
:100F700042A0B7005005200066A7B700A00A2000D5
:100F800066A7B70061E7A8000000000000000000AD
:100F90004200F9000060FE0000DB20001AA0B7004C
:100FA00000802200E40AB40014A0B70080002000F2
:100FB000ACAAB7000D409000004DBB001420EC001F
:100FC0001A20EC00AC2AED00FAFF3A0040A7A90075
:100FD0001000240060A7B7005005200066A7B700E6
:100FE000A00A200066A7B70061E7A8000000000083
:100FF0000000000061E7AF00FEFF370000002000A6
:1010000060A7B7000060FE001400F900030037007D
:1010100000C2B300616DB7006C6DEF0003003700D4
:1010200000C2B300616DB7006C6DEF004200F900C3
:1010300020C0B3006C4DB5006C003A0070C7B3001F
:10104000DF4AB50014003A004200F800000E20000C
:101050004200B70042A0B7001400F800D68ABF00D3
:1010600032A0B700D48ABF0014A0B700000420004B
:101070000AA0B700F0FF2F00000DBB00008DBB00E1
:1010800014A0EC000A20ED00FAFF3A001400F90069
:10109000DF6AEF004200F900D0CFB300DF4AB500AD
:1010A00017003A004200F800000E20004200B7008E
:1010B00042A0B7001400F80040A7A90010002400C7
:1010C00060A7B7005005200066A7B700A00A20005F
:1010D00066A7B70061E7A80000000000000000005C
:1010E00061E7AF00FEFF37000000200060A7B700F7
:1010F0000060FE001400F900DF6AEF004200F90012
:10110000E0CFB300DF4AB5001D003A004200F8000E
:10111000000E20004200B70042A0B7001400F80003
:10112000D68ABF0032A0B700D48ABF0014A0B7008F
:10113000000DBB002004240060A7B70040A7A90051
:101140004200F800000E20004200B70042A0B700A5
:101150005005200066A7B700A00A200066A7B700C8
:1011600061E7A80000000000000000004200F90054
:101170000060FE001400F900DF6AEF004200F90091
:1011800000C2B300EF4AB50018003A0000C0B30037
:10119000DF4AB50015003A004200F800000E2000BA
:1011A0004200B70042A0B7001400F800D68ABF0082
:1011B00032A0B700D48ABF0014A0B70000DB200023
:1011C0001AA0B7003D007800000DBB003D0078007C
:1011D000009DBB003D007800000DBB003D00780085
:1011E000009DBB001400F9004200F90054003700D4
:1011F00000C0B300ED4AB50007003A000400FC004F
:101200003B407800BDEAB700BDCABF0051020700ED
:10121000F9CABF00FA01070010C0B300ED4AB500DB
:101220000B003A000400FC003B407800BDEAB70028
:101230003B407800BEEAB700BDCABF0045020700C8
:10124000BECABF0043020700F8CABF00EC01070096
:1012500020C0B300ED4AB50013003A000800FC00BE
:101260003B407800BDEAB7003B407800BEEAB700DB
:101270003B407800BFEAB7003B407800C0EAB700C7
:10128000BDCABF0033020700BECABF00310207005B
:10129000BFCABF002F020700C0CABF002D0207004F
:1012A000F5CABF00D601070030C0B300ED4AB50053
:1012B00023003A001000FC003B407800BDEAB70074
:1012C0003B407800BEEAB7003B407800BFEAB70079
:1012D0003B407800C0EAB7003B407800C1EAB70065
:1012E0003B407800C2EAB7003B407800C3EAB70051
:1012F0003B407800C4EAB700BDCABF001502070032
:10130000BECABF0013020700BFCABF001102070018
:10131000C0CABF000F020700C1CABF000D0207000C
:10132000C2CABF000B020700C3CABF000902070000
:10133000C4CABF0007020700F4CABF00B00107001B
:101340000A409000FA4AB70057FD3A0062CDBF004C
:10135000020032008BCABF00FE0107004889BF00AF
:101360004CA9B70065FC37000020EF000220EF0019
:101370000420EF000620EF000820EF000A20EF0015
:101380000C20EF000E20EF001020EF001220EF00E5
:101390001420EF001620EF001820EF001A20EF00B5
:1013A0001C20EF0000DC20001EA0B70000E02000A1
:1013B00020A0B7000080200014A0B700F07F20001C
:1013C00002A0B70000002000004598001420EC00A7
:1013D0000220ED00FBFF3A003220EF004400A8009D
:1013E00083E0A90081E0A9008560A9009560A900BB
:1013F00000002700A820B70000002600A620B700A4
:10140000C0A2EF00C8A2EF0001E3A9002011210053
:1014100000A3B70000FE2F0002A3B70010102000A9
:101420000AA3B700100020000CA3B70001E3A80036
:10143000A00020009AAAB7006C0107009A2AED00CC
:10144000FDFF3A00E66AEF00CBA2AF0092EAA800E7
:10145000CBA2AE0092EAA900666DEF000000280062
:1014600020A2B7000040220022A2B7008540A900B8
:1014700042C7A90070002000A4A6B70030002000D9
:10148000D6E6B7000000200044A7B700E001200026
:1014900046A7B7000000280004A1B700F0FF2F0006
:1014A00000A1B7000001280010A1B700000028002B
:1014B00012A1B700800C20000EA1B7000068280020
:1014C00050A7B70080012000C4A2B70070FE2F0013
:1014D000C0A2B70000042100CCA2B70070382000E1
:1014E000C8A2B700100020009AAAB7003F01070069
:1014F0009A2AED00FDFF3A002682BF002202AF00CB
:10150000F8FF37002682BF002202AF00FDFF370040
:10151000B42AEF00B22AEF00C86AEF00C76AEF00F2
:10152000C66AEF00B7EAEF00E00020005CA9B70050
:10153000100020004CA9B7001000200040A9B700FF
:10154000A0002000BAAAB70092EAAE0076003700E9
:10155000A003200008A0B7003220EF000080220086
:101560000800B4001000BA0008A0B7000880BF004F
:1015700098A9B700C003200008A0B7003220EF00F0
:10158000008022000800B4001000BA0008A0B700D4
:101590000880BF009AA9B7002000200008A0B7006B
:1015A0003220EF00008022000800B4001000BA00D2
:1015B00008A0B70008C0BF0062EDB700000020001F
:1015C00008A0B7003220EF00008022000800B4001D
:1015D0001000BA0008A0B7000000200028A2B70041
:1015E00000C0B3000840B50002003A0030102000EF
:1015F00028A2B70010C0B3000840B50002003A00AE
:101600001008200028A2B70020C0B3000840B50091
:1016100002003A000004200028A2B70030C0B30046
:101620000840B50002003A00A002200028A2B7003E
:1016300040C0B3000840B50002003A00500120004D
:1016400028A2B70050C0B3000840B50002003A001D
:10165000A000200028A2B70060C0B3000840B50079
:1016600003003A005001200028A2B7002062A80021
:1016700070C0B3000840B50003003A00A00020008D
:1016800028A2B7002062A80080C0B3000840B500BF
:1016900002003A001000200028A2B70090C0B3005A
:1016A0000840B50002003A000000200028A2B70060
:1016B000A0C0B3000840B50003003A0010002000AD
:1016C00028A2B7002062A800B0C0B3000840B5004F
:1016D00003003A000000200028A2B7002062A80002
:1016E0008003200008A0B7003220EF000080220015
:1016F0000800B4001000BA0008A0B700800C200059
:101700000AA0B7000521B8000680BF0003003A0018
:101710000480BF0048A9B70002003700F0FF2F0087
:1017200048A9B70046003700F00F200062EDB7006F
:101730004000200008A0B7000000200028A2B70049
:1017400000C0B3000840B50002003A00301020008D
:1017500028A2B70010C0B3000840B50002003A004C
:101760001008200028A2B70020C0B3000840B50030
:1017700002003A000004200028A2B70030C0B300E5
:101780000840B50002003A00A002200028A2B700DD
:1017900040C0B3000840B50002003A0050012000EC
:1017A00028A2B70050C0B3000840B50002003A00BC
:1017B000A000200028A2B70060C0B3000840B50018
:1017C00003003A005001200028A2B7002062A800C0
:1017D00070C0B3000840B50003003A00A00020002C
:1017E00028A2B7002062A80080C0B3000840B5005E
:1017F00002003A001000200028A2B70090C0B300F9
:101800000840B50002003A000000200028A2B700FE
:10181000A0C0B3000840B50003003A00100020004B
:1018200028A2B7002062A800B0C0B3000840B500ED
:1018300003003A000000200028A2B7002062A800A0
:101840002222A9008560A9009560A80092EAAE0056
:1018500001003700EA013700E9FA37007EA9B70036
:101860007C09F9007609F9007609F8007C09F8008E
:1018700076A9ED007A29EC000010200078A9B700C5
:10188000004006007EA9B7007C09F9007609F9003E
:101890007609F8007C09F80076A9ED007A29EC00B9
:1018A0001000200078A9B700004006007EA9B7000C
:1018B0007C09F9007609F9007609F8007C09F8003E
:1018C00076A9ED007A29EC002000200078A9B70065
:1018D0008060A90040A7A800004006007EA9B700CC
:1018E0007C09F9007609F9007609F8007C09F8000E
:1018F00076A9ED007A29EC003000200078A9B70025
:1019000000DC20001EA0B7008040A90000400600B7
:101910007EA9B7007C09F9007609F9007609F8007C
:101920007C09F80076A9ED007A29EC00400020003F
:1019300078A9B7008080A900004006007EA9B70002
:101940007C09F9007609F9007609F8007C09F800AD
:1019500076A9ED007A29EC005000200078A9B700A4
:10196000E083BF007CA9B70080A0A900004006006A
:101970007EA9B7007C09F9007609F9007609F8001C
:101980007C09F80076A9ED007A29EC0060002000BF
:101990007CA9B700004006007EA9B7007C09F900C9
:1019A0007609F9007609F8007C09F80076A9ED00BF
:1019B0007A29EC00700020007CA9B70000400600E6
:1019C000D0C0B30001000700A0C0B3009EEAB7007A
:1019D0002222A9000060FE002322AF00FDFF370095
:1019E0009ECABF0024E2B700000006001041230099
:1019F00090A9B7009029ED00FEFF3A000000060014
:101A0000CDEAB700CECABF004220AE0007003700C3
:101A100016C0BF00CD4AB50016E0B70017C0BF0022
:101A2000FACAB50017E0B7000B00370000C0B300DA
:101A30006A4DB50005003A0016C0BF00E4EAB700E1
:101A400017C0BF00E5EAB700030037000020EF0031
:101A5000CDCABF00E02AB40000000600C6CABF001D
:101A600001003A00FDFF370000D72000B20AB400A1
:101A700018A0B700003020001C00600009003200F0
:101A8000CBCABF000700320000C4B300614DB700ED
:101A900061EDB7000500FC0000DC20001EA0B700CF
:101AA0009EFA37000C409000ECEAB7001820EC00DA
:101AB0000C409000B8EAB700C66AED00B2AAEC008C
:101AC000B2CAA900ECCABF0000000600C6CABF0027
:101AD00001003A00FDFF370000D72000B20AB40031
:101AE00018A0B700003020001C0060000900320080
:101AF000CBCABF000700320000C4B300614DB7007D
:101B000061EDB7000500FC0000DC20001EA0B7005E
:101B100082FA37000C409000ECEAB7001820EC0085
:101B20000C409000B8EAB700C66AED00B2AAEC001B
:101B3000B2CAA900ECCABF00ECCABF008CEAB6006A
:101B400000F020008C4AB4001040BA008CEAB700C4
:101B500000000600ECEAB700ECCABF009BFF0700DC
:101B6000ECCABF008BEAB60000F020008B4AB4003C
:101B70001040BA008BEAB70000000600D3FF070050
:101B8000ECCABF00005D7800000006008560A90077
:101B90000000F8001000F80026C2BF008AEAB70073
:101BA00000042000C64AB5001100320000D7200012
:101BB000B40AB40010A0B7008ACABF00004498005D
:101BC0001020EC0084E0AE000200370010C0B3002B
:101BD0000100370000C0B300004498000621EF0068
:101BE00084E0A900C66AEC00B4AAEC00B4CAA9005B
:101BF0002202AF00E8FF37001000F9000000F900F2
:101C0000004006000000F80094E0A900B7EAEF00E9
:101C100011E1A9000621EF000000F90084E0A9000D
:041C2000004006007A
:101E0000005E0000BCE20000613F0000DD830000D6
:101E1000C29C00007E200000A3FD00001F410000C6
:101E20009DC30000217F0000FCA20000401E0000B6
:101E30005F010000E3BD00003E60000082DC0000A6
:101E4000237D00009FC10000421C0000FEA0000096
:101E5000E1BF00005D03000080DE00003C62000086
:101E6000BEE00000025C0000DF810000633D000076
:101E70007C220000C09E00001D430000A1FF000066
:101E800046180000FAA40000277900009BC5000056
:101E900084DA000038660000E5BB00005907000046
:101EA000DB85000067390000BAE400000658000036
:101EB00019470000A5FB000078260000C49A000026
:101EC000653B0000D9870000045A0000B8E6000016
:101ED000A7F900001B450000C69800007A24000006
:101EE000F8A60000441A000099C70000257B0000F6
:101EF0003A64000086D800005B050000E7B90000E6
:101F00008CD20000306E0000EDB30000510F0000D5
:101F10004E100000F2AC00002F71000093CD0000C5
:101F2000114F0000ADF30000702E0000CC920000B5
:101F3000D38D00006F310000B2EC00000E500000A5
:101F4000AFF10000134D0000CE900000722C000095
:101F50006D330000D18F00000C520000B0EE000085
:101F6000326C00008ED00000530D0000EFB1000075
:101F7000F0AE00004C12000091CF00002D73000065
:101F8000CA94000076280000ABF500001749000055
:101F900008560000B4EA000069370000D58B000045
:101FA00057090000EBB50000366800008AD4000035
:101FB00095CB000029770000F4AA00004816000025
:101FC000E9B70000550B000088D60000346A000015
:101FD0002B75000097C900004A140000F6A8000005
:101FE000742A0000C8960000154B0000A9F70000F5
:101FF000B6E800000A540000D78900006B350000E5
:102000004440A8003420EF0060042000E0ECB7005A
:1020100020022000E1ECB700A0002000E2ECB700B5
:1020200000002000E3ECB70050042000D8ECB7001B
:10203000A0082000D9ECB70090002000DAECB7002F
:1020400060042000DBECB70060022000DCECB7008D
:10205000A0002000DDECB70000002000DEECB7009F
:10206000AA050700E0002000E7EAB700A000200072
:10207000BAAAB70000A025005EA9B700202620005C
:1020800060A9B700E0AF2C0068A9B700A05A2500EE
:102090006AA9B700002123006CA9B700406527009A
:1020A0006EA9B70080A92B0070A9B700C0ED2F0062
:1020B00072A9B70010002000B0A9B70000002000EE
:1020C000B2A9B700E00020005CA9B7001000200012
:1020D00074A9B7000000200082A9B70010002000FA
:1020E00084A9B700F0FF2F0088A9B700F0FF2F00E8
:1020F00086A9B7003220EF00808722001000BA00C6
:1021000022AAB700A08722001000BA0024AAB700B4
:1021100083E0A8002682BF002202AF00FDFF370047
:10212000B42AEF00B22AEF00C86AEF00C76AEF00D6
:10213000C66AEF00B7EAEF008560A9009560A800C5
:102140008760A9008500A9009500A800A0002000D4
:102150009AAAB700B30407009A2AED00FDFF3A00DF
:102160000060FE0040A7A80093EAA9002003200019
:102170009AAAB700AB0407009A2AED00FDFF3A00C7
:102180002062AE00030037000000200010A1B7005D
:1021900011E1A800CC82A900CD42A800C462A90028
:1021A000CD62A900007D200008A0B700CCA2A80045
:1021B00000000000CCA2A9000820ED00FBFF3A00BF
:1021C000C462A800CD62A800800C20000EA1B70058
:1021D0000000200000A3B7002011210000A3B700D9
:1021E00001E3A8003220EF0000C0B300ECEAB70022
:1021F00060EDB70061EDB7006AEDB70066EDB700BE
:10220000CCEAB700FAEAB70010002000F9EAB700FC
:1022100020002000F8EAB70030002000F7EAB700FD
:1022200040002000F5EAB70080002000F4EAB70083
:10223000F0CFB300F3EAB700B7EAB700800220009E
:102240006BEDB700800F2000F2EAB700100020000D
:10225000F1EAB700B0002000F0EAB700000C20005F
:10226000D3EAB70080002000DDEAB700B00020000C
:10227000DCEAB70000002000E4EAB700000020001C
:10228000E5EAB70000002000E0EAB7000000200007
:10229000E1EAB700C0FE2000EAAAB7002882BF002A
:1022A0000020EC002062AF00020037004100DD009A
:1022B000010037004200DD0064AAB7000020EF00F3
:1022C0006BCDBF00BA0AB400640ABC000680BF0030
:1022D00003003A000480BF000CA1B70001003700E2
:1022E0000CA1EF00007D20002AAAB7002C2AEC00E8
:1022F00061CDBF0002003A00C482A900000037008F
:1023000000E0200014A0B700CB6AEF008C6AEF0059
:10231000E96AEF00A4040700ECCABF0088EAB7002E
:1023200010C0B300B84AB50003003A0000CCB300B7
:10233000EC4AB600060037000020EF00C9CABF0013
:1023400003003200C96AEF0000CCB300EC4AB600CB
:10235000EEFF3200CBEAEF00F0C1B300884AB600CE
:10236000D2EAB70000CCB300884AB600D3EAB7007F
:1023700000CCB300D34AB50004003A00F0CFB3005C
:10238000884AB50001003A00DDFF370000C8B300FD
:10239000D34AB50027003A00D0CBB300884AB50035
:1023A0000E003A0040C0B300664DB5000500310094
:1023B0000020EF0066CDBF000020B40016A0B700DB
:1023C000010037000B002000C4E9EF008E89BF0038
:1023D0001620B4000B00900000400100F0C3B300D1
:1023E000884AB600D1EAB700E9EAEF00D1CABF00D7
:1023F0004200A90000C0D60000C0D60000C0D60030
:1024000000C0D60017E0B70000C0D700F24AB600FF
:1024100016E0B70017C0BF00F14AB600F04AB4009A
:1024200017E0B700C4E9EF003B40780088EAB70046
:102430000000370088CABF00005D780000CCB30000
:10244000884AB600D3EAB700F0C3B300884AB600A2
:10245000D1EAB70080C0B300884AB600CEEAB70020
:1024600040C0B300884AB600EEEAB70030C0B300FF
:10247000884AB600EDEAB70000C2B300884AB60049
:10248000EFEAB70000CCB300D34AB5000A003A0027
:1024900000C2B300EF4AB50007003A0000C0B30025
:1024A000E94AB500030032000B409000005D78005F
:1024B000010037009104070000C4B300D34AB500FF
:1024C00065003A0040C0B300EE4AB5000A003A0089
:1024D00000C0B300E94AB500050032003B40780077
:1024E000005D78003B407800005D78000200370016
:1024F000820407008104070000C2B300EF4AB50060
:1025000055003A0000C0B300ED4AB5000A003A0099
:1025100000C1B300884AB6000600320000C0B30014
:10252000E94AB500020032003B407800005D7800C7
:10253000010037007104070010C0B300ED4AB50078
:102540000D003A0000C1B300884AB600080032000E
:1025500000C0B300E94AB500040032003B407800F7
:10256000005D78003B407800005D78000200370095
:10257000620407006104070020C0B300ED4AB50003
:1025800013003A0000C1B300884AB6000C003200C4
:1025900000C0B300E94AB500080032003B407800B3
:1025A000005D78003B407800005D78003B4078009B
:1025B000005D78003B407800005D78000400370043
:1025C0004E0407004D0407004C0407004B040700AD
:1025D00030C0B300ED4AB5001F003A0000C1B3009F
:1025E000884AB6001400320000C0B300E94AB500C2
:1025F000100032003B407800005D78003B407800DE
:10260000005D78003B407800005D78003B4078003A
:10261000005D78003B407800005D78003B4078002A
:10262000005D78003B407800005D78003B4078001A
:10263000005D780008003700300407002F04070011
:102640002E0407002D0407002C0407002B040700AC
:102650002A0407002904070000C0B300E94AB500B6
:1026600002003A0000C0B30088EAB70000C0B3001F
:102670000045980000C0B300E94AB5000A003200E6
:102680003B40780088EAB700005D780014C0BF00C6
:10269000EA4AB50015C0BF00EBCAB5000200310020
:1026A00000C1B300616DB70088CABF0063FF3A0084
:1026B000E96AEF0000C0B3000045980062CDBF009A
:1026C000090032008CCABF0072030700ECCABF00C9
:1026D0008C4AB5000400320010C0B300616DB70031
:1026E000636DEC0006FF3700CB6AEF0000E02000CE
:1026F00014A0B7008B6AEF003A40780088EAB70070
:1027000000CCB300884AB600D3EAB70080C0B3005B
:10271000884AB600CEEAB70040C0B300884AB60087
:10272000EEEAB70030C0B300884AB600EDEAB70061
:1027300000C2B300884AB600EFEAB70000CCB3008D
:10274000D34AB500F0003A00F0C1B300884AB600A1
:10275000D2EAB70000C2B300884AB600EFEAB70079
:1027600016C0BF00E2EAB70017C0BF00E3EAB70037
:1027700000C1B300D24AB5002A00310000D62000C3
:1027800016A0B70016C0BF00D24AB40016E0B700CA
:1027900017C0BF00FACAB40017E0B70000C2B30008
:1027A000EF4AB5001C003A003A4078008045980096
:1027B000B0CEB300884AB50012003A002882BF00AC
:1027C0000020EC002062AF00020037004100DD0075
:1027D000010037004200DD0064AAB7000020EF00CE
:1027E0006BCDBF00BA0AB400640ABC000680BF000B
:1027F00003003A000480BF000CA1B70001003700BD
:102800000CA1EF0060CEB300884AB50001003A0089
:10281000BE030700020037000B409000AD03070025
:10282000B500370000C2B300EF4AB50042003A00DD
:1028300070CFB300884AB50002003A003A407800F1
:102840003C00370080CFB300884AB50009003A0049
:1028500000C0B3006A4DB50003003A003A4078006A
:10286000E4EAB700020037003A407800E0EAB70037
:102870003000370090CFB300884AB50009003A0015
:1028800000C0B3006A4DB50003003A003A4078003A
:10289000E5EAB700020037003A407800E1EAB70005
:1028A00024003700A0CFB300884AB50011003A00D9
:1028B00000C0B3006A4DB50007003A003A40780006
:1028C000E44AB400E4EAB700E5CABF00FACAB400BB
:1028D000E5EAB700060037003A407800E04AB40065
:1028E000E0EAB700E1CABF00FACAB400E1EAB70003
:1028F00010003700D0CFB300884AB50003003A007B
:102900003A407800CCEAB7000A003700E0CFB300C5
:10291000884AB50007003A003A407800ECEAB70070
:10292000A0C5B300EC4AB50001003A00B4FD370081
:10293000000037007000370000CDB300884AB500B2
:1029400003003A0070C3B300620307006A00370057
:1029500010CDB300884AB50003003A0090C4B3001C
:102960005C0307006400370020CDB300884AB5003F
:1029700003003A0070C3B300560307005E0037003F
:1029800030CDB300884AB50003003A0070C3B300ED
:10299000500307005800370040CDB300884AB50007
:1029A00003003A00D0C0B3004A03070052003700CA
:1029B00050CDB300884AB50003003A00E7CABF0013
:1029C000440307004C00370060CDB300884AB500CF
:1029D00003003A00E6CABF003E0307004600370086
:1029E00070CDB300884AB50003003A0040C9BF006B
:1029F0003803070040003700A0CDB300884AB50077
:102A000003003A0000C0B300320307003A00370069
:102A1000B0CDB300884AB50003003A007BCDBF00BB
:102A20002C03070034003700D0CDB300884AB5002E
:102A300003003A0000C0B300260307002E00370051
:102A4000E0CDB300884AB50003003A0020C0B300CF
:102A50002003070028003700C0CDB300884AB50026
:102A600003003A0080C0B3001A03070022003700B9
:102A7000C0CDB300884AB50003003A0080C0B3005F
:102A8000140307001C00370080CDB300884AB5004E
:102A900008003A0000C0B3006A4DB50002003A00D9
:102AA000E4CABF0001003700E0CABF000903070005
:102AB0001100370090CDB300884AB50008003A00F5
:102AC00000C0B3006A4DB50002003A00E5CABF007D
:102AD00001003700E1CABF00FE0207000600370010
:102AE000F0CDB300884AB50003003A00A0C5B3009A
:102AF000F802070000003700E2CABF0016E0B70086
:102B0000E3CABF0017E0B700F0C3B300884AB600BD
:102B1000D1EAB70000C4B300D34AB500CE013A00F1
:102B200040C0B300EE4AB5000C003A0000C0B3004C
:102B30006A4DB50005003A003A407800E4EAB70073
:102B40003A407800E5EAB700040037003A407800E0
:102B5000E0EAB7003A407800E1EAB70000C0B3000D
:102B60006A4DB50005003A00E4CABF0016E0B700A0
:102B7000E5CABF0017E0B70005003700E0CABF0094
:102B800016E0B700E1CABF00F04AB40017E0B70092
:102B900020C0B3006C4DB50002003A004200A9000D
:102BA0000600370000C0B3006A4DB50002003A00CD
:102BB0004200A900010037004200A90004003900CA
:102BC00000DB200016A0B70000C2B300616DB700A3
:102BD00010C0B3006C4DB50016003A003220EF0073
:102BE0004200F800000E20004200B70042A0B700EB
:102BF00000DB20001AA0B70000802200E44AB400E5
:102C000018A0B70080002000ACAAB7001880BF0051
:102C10001040BA00804698001820EC001A20EC0002
:102C2000AC2AED00F9FF3A0000DB200016A0B70047
:102C30004200F90020C0B3006C4DB50034003A00EA
:102C400080002000DDEAB700B0002000DCEAB70019
:102C50004200A900DA8ABF000080D700D6AAB700D8
:102C6000D88ABF000080D7000000A900D4AAB7000E
:102C7000F0FF2700E40AB6004200A9000080D70058
:102C80000000A900D40AB400D4AAB70000C8B30059
:102C9000E54AB6001B003A0000DB200016A0B70092
:102CA00000C2B300EF4AB500150032001400F8006E
:102CB000D68ABF0032A0B700D48ABF0014A0B700E4
:102CC00000DB20001AA0B7001480BF001000BA007B
:102CD000801E78001480BF001080BA00801E78002B
:102CE00014A0EC001480BF001000BA00801E780011
:102CF0001480BF001080BA00801E78001400F90014
:102D00000300370080AD2000E44AB40016A0B700ED
:102D100000C2B300EF4AB500FB003A0000C0B300A8
:102D2000ED4AB50004003A003A407800805D780032
:102D3000F9CABF00C001070010C0B300ED4AB500DA
:102D400007003A000400FC003A407800805D7800FB
:102D50003A407800805D7800F8CABF00B6010700ED
:102D600020C0B300ED4AB5000B003A000800FC009B
:102D70003A407800805D78003A407800805D7800C5
:102D80003A407800805D78003A407800805D7800B5
:102D9000F5CABF00A801070030C0B300ED4AB50076
:102DA00013003A001000FC003A407800805D780083
:102DB0003A407800805D78003A407800805D780085
:102DC0003A407800805D78003A407800805D780075
:102DD0003A407800805D78003A407800805D780065
:102DE0003A407800805D7800F4CABF009201070085
:102DF0008602070010C0B3006C4DB50052003A00C7
:102E00003220EF004200F800000E20004200B70020
:102E100042A0B700E5CABF0047003A0000C8B300AF
:102E2000E44AB60040003A001400F8000080220096
:102E300014A0B70000042000ACAAB7001480BF00A3
:102E40001000BA00000DBB0000002000008DBB0088
:102E500014A0EC00AC2AED00F8FF3A003220EF009D
:102E60002004240060A7B7000080220014A0B7004F
:102E70001000BA00000DBB0040A7A9004200F800F6
:102E8000000E20004200B70042A0B700500520000D
:102E900066A7B700A00A200066A7B70061E7A800F0
:102EA00000000000000000004200F9000060FE0089
:102EB00000DB20001AA0B70000802200E40AB40062
:102EC00014A0B70080002000ACAAB7000D4090000D
:102ED000004DBB001420EC001A20EC00AC2AED00E1
:102EE000FAFF3A0040A7A9001000240060A7B7002D
:102EF0005005200066A7B700A00A200066A7B7000B
:102F000061E7A800000000000000000061E7AF00DA
:102F1000FEFF37000000200060A7B7000060FE0041
:102F20001400F9000300370000C2B300616DB70060
:102F30006C6DEF000300370000C2B300616DB70095
:102F40006C6DEF004200F90020C0B3006C4DB5007D
:102F50006C003A0070C7B300DF4AB50014003A00B5
:102F60004200F800000E20004200B70042A0B70067
:102F70001400F800D68ABF0032A0B700D48ABF0080
:102F800014A0B700000420000AA0B700F0FF2F0033
:102F9000000DBB00008DBB0014A0EC000A20ED006A
:102FA000FAFF3A001400F900DF6AEF004200F9006E
:102FB000D0CFB300DF4AB50017003A004200F80056
:102FC000000E20004200B70042A0B7001400F80035
:102FD00040A7A9001000240060A7B70050052000FA
:102FE00066A7B700A00A200066A7B70061E7A8009F
:102FF000000000000000000061E7AF00FEFF3700A6
:103000000000200060A7B7000060FE001400F90077
:10301000DF6AEF004200F900E0CFB300DF4AB500FD
:103020001D003A004200F800000E20004200B700E8
:1030300042A0B7001400F800D68ABF0032A0B70043
:10304000D48ABF0014A0B700000DBB0020042400E8
:1030500060A7B70040A7A9004200F800000E2000BA
:103060004200B70042A0B7005005200066A7B70095
:10307000A00A200066A7B70061E7A80000000000D2
:10308000000000004200F9000060FE001400F9009A
:10309000DF6AEF004200F90000C2B300EF4AB5005A
:1030A00018003A0000C0B300DF4AB50015003A002E
:1030B0004200F800000E20004200B70042A0B70016
:1030C0001400F800D68ABF0032A0B700D48ABF002F
:1030D00014A0B70000DB20001AA0B7003D00780064
:1030E000000DBB003D007800009DBB003D00780056
:1030F000000DBB003D007800009DBB001400F900EE
:103100004200F9005400370000C0B300ED4AB5009A
:1031100007003A000400FC003B407800BDEAB7001D
:10312000BDCABF006B010700F9CABF00C20007009B
:1031300010C0B300ED4AB5000B003A000400FC00DB
:103140003B407800BDEAB7003B407800BEEAB700DC
:10315000BDCABF005F010700BECABF005D01070016
:10316000F8CABF00B400070020C0B300ED4AB500A4
:1031700013003A000800FC003B407800BDEAB700AD
:103180003B407800BEEAB7003B407800BFEAB7009A
:103190003B407800C0EAB700BDCABF004D01070040
:1031A000BECABF004B010700BFCABF0049010700EC
:1031B000C0CABF0047010700F5CABF009E00070054
:1031C00030C0B300ED4AB50023003A001000FC0007
:1031D0003B407800BDEAB7003B407800BEEAB7004C
:1031E0003B407800BFEAB7003B407800C0EAB70038
:1031F0003B407800C1EAB7003B407800C2EAB70024
:103200003B407800C3EAB7003B407800C4EAB7000F
:10321000BDCABF002F010700BECABF002D010700B5
:10322000BFCABF002B010700C0CABF0029010700A9
:10323000C1CABF0027010700C2CABF00250107009D
:10324000C3CABF0023010700C4CABF002101070091
:10325000F4CABF00780007000A409000FA4AB7009D
:1032600025FD3A0062CDBF00020032008BCABF00CC
:10327000180107004889BF004CA9B700C9EAEF0050
:10328000C4C9BF000200320060010700C469EF003A
:1032900014FC37007EA9B7007C09F9007609F90013
:1032A0007609F8007C09F80076A9ED007A29EC008F
:1032B0000010200078A9B700004006007EA9B700E2
:1032C0007C09F9007609F9007609F8007C09F80014
:1032D00076A9ED007A29EC001000200078A9B7004B
:1032E000004006007EA9B7007C09F9007609F900C4
:1032F0007609F8007C09F80076A9ED007A29EC003F
:103300002000200078A9B7008060A90040A7A8008D
:10331000004006007EA9B7007C09F9007609F90093
:103320007609F8007C09F80076A9ED007A29EC000E
:103330003000200078A9B70000DC20001EA0B700F4
:103340008040A900004006007EA9B7007C09F90072
:103350007609F9007609F8007C09F80076A9ED00F5
:103360007A29EC004000200078A9B7008080A900ED
:10337000004006007EA9B7007C09F9007609F90033
:103380007609F8007C09F80076A9ED007A29EC00AE
:103390005000200078A9B700E083BF007CA9B700E7
:1033A00080A0A900004006007EA9B7007C09F900B2
:1033B0007609F9007609F8007C09F80076A9ED0095
:1033C0007A29EC00600020007CA9B70000400600CC
:1033D0007EA9B7007C09F9007609F9007609F800A2
:1033E0007C09F80076A9ED007A29EC007000200035
:1033F0007CA9B70000400600D0C0B3000100070060
:10340000A0C0B3009EEAB7002222A9000060FE001F
:103410002322AF00FDFF37009ECABF0024E2B700A1
:10342000000006001041230090A9B7009029ED008C
:10343000FEFF3A0000000600CDEAB700CECABF008A
:103440004220AE000700370016C0BF00CD4AB500CD
:1034500016E0B70017C0BF00FACAB50017E0B70002
:103460000B00370000C0B3006A4DB50005003A00FC
:1034700016C0BF00E4EAB70017C0BF00E5EAB70016
:10348000030037000020EF00CDCABF00E02AB400DF
:1034900000000600C6CABF002A003A004289BF00E9
:1034A00008003200100320004009B600030032007B
:1034B0005029EF005229EF00D40007004229EF0005
:1034C000542AEF00528ABF00070032000028EF00A4
:1034D0000228EF00CD000700CC00070050A9EF0044
:1034E00052A9EF00522AEF00C462A900F2000700BF
:1034F000CB02AF00160AA800CB02AE00160AA90044
:10350000C462A800CD62A900EB000700CB02AF00A7
:10351000162AA800CB02AE00162AA900CD62A80088
:1035200060662600180ABC000680BF00E4A9B70048
:1035300090992900180ABC000680BF00E6A9B700D0
:10354000D4FF370000D72000B20AB40018A0B7009B
:10355000003020001C00600009003200CBCABF0010
:103560000700320000C4B300614DB70061EDB70041
:103570000500FC0000DC20001EA0B70060FB370047
:103580000C409000ECEAB7001820EC000C409000D2
:10359000B8EAB700C66AED00B2AAEC00B2CAA90048
:1035A000ECCABF0000000600C6CABF002A003A00ED
:1035B0004289BF0008003200100320004009B60015
:1035C000030032005029EF005229EF008F0007005E
:1035D0004229EF00542AEF00528ABF000700320050
:1035E0000028EF000228EF0088000700870007008E
:1035F00050A9EF0052A9EF00522AEF00C462A900BF
:10360000AD000700CB02AF00160AA800CB02AE0047
:10361000160AA900C462A800CD62A900A60007008E
:10362000CB02AF00162AA800CB02AE00162AA900D2
:10363000CD62A80060662600180ABC000680BF00A4
:10364000E4A9B70090992900180ABC000680BF00C1
:10365000E6A9B700D4FF370000D72000B20AB400B3
:1036600018A0B700003020001C00600009003200E4
:10367000CBCABF000700320000C4B300614DB700E1
:1036800061EDB7000500FC0000DC20001EA0B700C3
:103690001BFB37000C409000ECEAB7001820EC0050
:1036A0000C409000B8EAB700C66AED00B2AAEC0080
:1036B000B2CAA900ECCABF00ECCABF008CEAB600CF
:1036C00000F020008C4AB4001040BA008CEAB70029
:1036D00000000600ECEAB700ECCABF0049FF070093
:1036E000ECCABF008BEAB60000F020008B4AB400A1
:1036F0001040BA008BEAB70000000600AAFF0700DE
:10370000ECCABF00005D78000000060040C0B300B6
:10371000664DB500060031000020EF0066CDBF0009
:103720000020B4000020B4000CA0B7000100370056
:103730000600200040602A000C20B4000600900023
:1037400026AAB7000CA0EC00060090008AA9B700DA
:10375000E0512A0028AAB70040612A008EA9B700CC
:1037600000000600000020008B49B4008CA9B700BF
:103770008CC9BF0003003200E0FF07008C29ED0078
:10378000FBFF370062CDBF000C0032008CCABF00C7
:1037900040FF0700ECCABF008C4AB50007003200AA
:1037A00010C0B300616DB700636DEC000500FC0054
:1037B00000DC20001EA0B700D1FA37008B6AEF00B2
:1037C00000E0200014A0B700000006008CA9B7009C
:1037D0008CC9BF00040032003B407800BDFF0700E9
:1037E0008C29ED00FAFF3700000006008CA9B70015
:1037F0008CC9BF00040032003A407800805D780038
:103800008C29ED00FAFF3700000006005089BF0048
:103810000028B6005289BF000228B60000C8BF00C9
:1038200030EAB700316AEF00CD62A900220007003C
:10383000B6020700CD62A8002FEAAF00160AA80062
:103840002FEAAE00160AA9002E8ABF0010EAB700C0
:1038500001C8BF0030EAB700316AEF00C462A900B6
:1038600015000700A9020700C462A8002FEAAF00F4
:10387000162AA8002FEAAE00162AA9002E8ABF0039
:1038800011EAB700108ABF0000A0EE005029B60070
:10389000128ABF0000A0EE005229B600160AAE0040
:1038A000010037005069EF00162AAE000100370012
:1038B0005169EF0000000600000006000000000053
:1038C0000000000000000000000006008560A90064
:1038D0000000F8001000F80026C2BF008AEAB70016
:1038E00000042000C64AB5001100320000D72000B5
:1038F000B40AB40010A0B7008ACABF000044980000
:103900001020EC0084E0AE000200370010C0B300CD
:103910000100370000C0B300004498000621EF000A
:1039200084E0A900C66AEC00B4AAEC00B4CAA900FD
:103930002202AF00E8FF37001000F9000000F90094
:10394000004006000000F8000000F9008C20A900EB
:10395000004006000000F80094E0A900B7EAEF007C
:1039600011E1A9000000F90084E0A9000040060070
:103970000060FE000000F8002A8ABF000800320044
:103980002A2AED0002003A00F01F20002CAAB700FE
:103990002D2AAF00C482A9002D2AAE00C482A8003F
:1039A0004889BF004A09BD00020032004889BF00B3
:1039B0004CA9B7004C89BF00040032004C29ED002F
:1039C00002003A00100020004029B7004889BF00DB
:1039D0004AA9B70000CF2100E009B400004001006F
:1039E000080037004500370080003700BB00370073
:1039F000F6003700270137005801370089013700EA
:103A0000B9013700C3E2A800CDC2A800CDA2A90029
:103A1000CC62A80025C3BF0010E8B70027C3BF00D1
:103A200018E8B70021C3BF0020E8B70023C3BF00D8
:103A300028E8B700C3E2A9000AA3A8000BA3A800C6
:103A4000E7C9BF001048B500020039000808A80007
:103A500004003700E5C9BF001048B500010031007F
:103A60000808A900E7C9BF001848B50002003900DE
:103A70000908A80004003700E5C9BF001848B500D0
:103A8000010031000908A90030C0B300664DB5003F
:103A900007003A0010C1B3002048B5000200390009
:103AA0000A08A800010037000A08A9000900370029
:103AB000E7C9BF002048B500020039000A08A80085
:103AC00004003700E5C9BF002048B50001003100FF
:103AD0000A08A900E7C9BF002848B500020039005C
:103AE0000B08A80004003700E5C9BF002848B5004E
:103AF000010031000B08A90000023700CDC2A90067
:103B0000CDA2A800CC62A80025C3BF0011E8B70071
:103B100027C3BF0019E8B70021C3BF0021E8B700E1
:103B200023C3BF0029E8B7000AA3A8000BA3A8007D
:103B3000E7C9BF001148B500020039000828A800F5
:103B400004003700E5C9BF001148B500010031008D
:103B50000828A900E7C9BF001948B50002003900CC
:103B60000928A80004003700E5C9BF001948B500BE
:103B7000010031000928A90030C0B300664DB5002E
:103B800007003A0010C1B3002148B5000200390017
:103B90000A28A800010037000A28A90009003700F8
:103BA000E7C9BF002148B500020039000A28A80073
:103BB00004003700E5C9BF002148B500010031000D
:103BC0000A28A900E7C9BF002948B500020039004A
:103BD0000B28A80004003700E5C9BF002948B5003C
:103BE000010031000B28A900C4013700CDC2A80094
:103BF000CDA2A800CC62A80025C3BF0012E8B70080
:103C000027C3BF001AE8B70021C3BF0022E8B700EE
:103C100023C3BF002AE8B7000AA3A8000BA3A8008B
:103C2000E7C9BF001248B500020039000848A800E3
:103C300004003700E5C9BF001248B500010031009B
:103C40000848A900E7C9BF001A48B50002003900BA
:103C50000948A80004003700E5C9BF001A48B500AC
:103C6000010031000948A90030C0B300664DB5001D
:103C700007003A0010C1B3002248B5000200390025
:103C80000A48A800010037000A48A90009003700C7
:103C9000E7C9BF002248B500020039000A48A80061
:103CA00004003700E5C9BF002248B500010031001B
:103CB0000A48A900E7C9BF002A48B5000200390038
:103CC0000B48A80004003700E5C9BF002A48B5002A
:103CD000010031000B48A90088013700CDC2A900BE
:103CE000CDA2A900CC62A90025C3BF0013E8B7008C
:103CF00027C3BF001BE8B70021C3BF0023E8B700FC
:103D000023C3BF002BE8B7000AA3A8000BA3A80099
:103D1000E7C9BF001348B500020039000868A800D1
:103D200004003700E5C9BF001348B50001003100A9
:103D30000868A900E7C9BF001B48B50002003900A8
:103D40000968A80004003700E5C9BF001B48B5009A
:103D5000010031000968A90030C0B300664DB5000C
:103D600007003A0010C1B3002348B5000200390033
:103D70000A68A800010037000A68A9000900370096
:103D8000E7C9BF002348B500020039000A68A8004F
:103D900004003700E5C9BF002348B5000100310029
:103DA0000A68A900E7C9BF002B48B5000200390026
:103DB0000B68A80004003700E5C9BF002B48B50018
:103DC000010031000B68A9004C013700CDC2A800EA
:103DD000CDA2A900CC62A90025C3BF0014E8B7009A
:103DE00027C3BF001CE8B70021C3BF0024E8B70009
:103DF00023C3BF002CE8B7000AA3A8000BA3A800A8
:103E0000E7C9BF001448B500020039000888A800BF
:103E100004003700E5C9BF001448B50001003100B7
:103E20000888A900E7C9BF001C48B5000200390096
:103E30000988A80004003700E5C9BF001C48B50088
:103E4000010031000988A900E7C9BF002448B50076
:103E5000020039000A88A80004003700E5C9BF0045
:103E60002448B500010031000A88A900E7C9BF0055
:103E70002C48B500020039000B88A8000400370068
:103E8000E5C9BF002C48B500010031000B88A9002E
:103E90001A013700CDC2A900CDA2A800CC62A900AA
:103EA00025C3BF0015E8B70027C3BF001DE8B70052
:103EB00021C3BF0025E8B70023C3BF002DE8B7002A
:103EC0000AA3A8000BA3A800E7C9BF001548B500C6
:103ED0000200390008A8A80004003700E5C9BF00A7
:103EE0001548B5000100310008A8A900E7C9BF00C6
:103EF0001D48B5000200390009A8A80004003700D9
:103F0000E5C9BF001D48B5000100310009A8A9009E
:103F1000E7C9BF002548B500020039000AA8A8007B
:103F200004003700E5C9BF002548B5000100310095
:103F30000AA8A900E7C9BF002D48B5000200390052
:103F40000BA8A80004003700E5C9BF002D48B50044
:103F5000010031000BA8A900E8003700CDC2A8007D
:103F6000CDA2A800CC62A90025C3BF0016E8B70007
:103F700027C3BF001EE8B70021C3BF0026E8B70073
:103F800023C3BF002EE8B7000AA3A8000BA3A80014
:103F9000E7C9BF001648B5000200390008C8A800EC
:103FA00004003700E5C9BF001648B5000100310024
:103FB00008C8A900E7C9BF001E48B50002003900C3
:103FC00009C8A80004003700E5C9BF001E48B500B5
:103FD0000100310009C8A900E7C9BF002648B500A3
:103FE000020039000AC8A80004003700E5C9BF0074
:103FF0002648B500010031000AC8A900E7C9BF0082
:104000002E48B500020039000BC8A8000400370094
:10401000E5C9BF002E48B500010031000BC8A9005A
:10402000B6003700CDC2A900CDA2A900CC62A8007D
:1040300025C3BF0017E8B70027C3BF001FE8B700BC
:1040400021C3BF0027E8B70023C3BF002FE8B70094
:104050000CA3A800E7C9BF001748B500020039004B
:1040600008E8A80004003700E5C9BF001748B500FC
:104070000100310008E8A900E7C9BF001F48B500EA
:104080000200390009E8A80004003700E5C9BF00B4
:104090001F48B5000100310009E8A900E7C9BF00C9
:1040A0002748B500020039000AE8A80004003700DC
:1040B000E5C9BF002748B500010031000AE8A900A2
:1040C000E7C9BF002F48B500020039000BE8A8007F
:1040D00004003700E5C9BF002F48B50001003100DA
:1040E0000BE8A900850037002883BF0018AAB70095
:1040F0000AA3A8000BA3A80067CDBF0006003200EA
:104100004689BF0004003A004029EF00542AEF001E
:104110004229EF0052AAEF0040C32100180ABD0057
:104120000400390016EAA800000220004029B70068
:104130000300370016EAA900F0FD2F004029B60061
:10414000001A2E00180ABD000400310017EAA8006A
:10415000000120004029B7000300370017EAA9003A
:10416000F0FE2F004029B600108ABF00120AB700E7
:1041700002003200800020004029B7000020EF003C
:104180000000A900160AAF000000A8000020A90046
:10419000162AAF000020A8000080BF0002003200F5
:1041A000400020004029B70040C0B300664DB50074
:1041B00002003900000420004029B7004089BF00F8
:1041C00002003A00CDE2A8000C00370010032000E6
:1041D0004009B600040032005029EF005229EF00D8
:1041E0004268EF004028EF00CDE2A900548ABF00EA
:1041F00002003A0042A9EF0054AAEF00528ABF0021
:1042000003003A004689BF0001003200676DEF00ED
:1042100067CDBF0046E9B70030C0B300664DB500BA
:1042200034003A009229A9000A08AF009229A80098
:104230009249A9009609AF009249A8009269A90085
:104240000A28AF009269A8009289A9009629AF00B8
:104250009289A800001B2A009209B4000EA0B700A2
:104260009889BF004500DD000E20B40007009000D3
:10427000A029B4009229A9000A48AF009229A800F9
:104280009249A9009649AF009249A8009269A900F5
:104290000A68AF009269A8009289A9009669AF00E8
:1042A0009289A800001B2A009209B4000EA0B70052
:1042B0009A89BF004500DD000E20B4000700900081
:1042C000A229B4009609A9000A08AF009609A8001F
:1042D0009629A9000A28AF009629A8009649A900A6
:1042E0000A48AF009649A8009669A9000A68AF007D
:1042F0009669A800E029EF0001003700E0A9EC0072
:104300000000F9008500A90000400600000120001F
:104310003AAAB700CCA2A800300AAF00CC82A8000D
:10432000300AAE00CC82A90064FD0700CCA2A9002F
:104330002FEAA900CB02AF002FEAA800308ABF0005
:104340004100DE0030AAB7002E8ABF004100DE0027
:104350002EAAB7003A2AED00EEFF3A000000060050
:104360000000000001000000FFFF0000000000004E
:10437000000000000000FF000000FF00000000003F
:1043800000000000000000000000FF00000000002E
:10439000000000000000000000000000000000001D
:1043A00000000000FFFF000001000000000000000E
:1043B000000000000000FF000000FF0000000000FF
:1043C000000000000000FF000000FF0000000000EF
:1043D00000000000000000000000000000000000DD
:1043E00000000000010000000000000000000000CC
:1043F000FFFF00000000FF000000000000000000C0
:10440000000000000000FF000000FF00FFFF0000B0
:10441000000000000000000001000000000000009B
:1044200000000000FFFF000000000000000000008E
:10443000010000000000FF0000000000000000007C
:10444000000000000000FF000000FF00010000006D
:104450000000000000000000FFFF0000000000005E
:104460000000000001000000FFFF0000000000004D
:10447000FFFF00000000FF000000FF00010000003F
:10448000010000000000FF000000FF00FFFF00002F
:1044900000000000FFFF000001000000000000001D
:1044A00000000000FFFF000001000000000000000D
:1044B000010000000000FF000000FF00FFFF0000FF
:1044C000FFFF00000000FF000000FF0001000000EF
:1044D0000000000001000000FFFF000000000000DD
:1044E000B00000000000000053740000616E000086
:1044F000646100007264000000000000B000000071
:1045000001000000496E000070750000745F00003B
:104510004F7500007470000075740000000000000A
:10452000B001000001000000494F00005F410000A1
:104530006E6100006C6F000067000000B0020000B8
:1045400001000000494F00005F4100006E61000063
:104550006C6F0000675F000046690000656C00003A
:10456000645600006F6C0000746100006765000015
:1045700000000000B003000001000000494F0000EF
:104580005F4500006E6300006F640000657200000C
:104590005F4100006E6100006C6F0000675F00000B
:1045A00046690000656C0000647600006F6C0000D6
:1045B000746100006765000000000000A02000009A
:1045C00001000000000000000000000000000000EA
:1045D00000000000080800004E6F00006E6500003B
:1045E000004900006E7000007574000000000000BB
:1045F000A01000000180000000000000000000008A
:104600000000000000000000000800004E6F0000E5
:104610006E650000004F00007574000070750000AA
:1046200074000000A008000002000000000000006C
:1046300000000000333300001142000010080000A9
:10464000566F00006C74000073000000416E0000A3
:10465000616C00006F670000496E000030000000D0
:10466000A0080000020000000000000000000000A0
:10467000333300001142000011080000566F0000A3
:104680006C74000073000000416E0000616C00005B
:104690006F670000496E000031000000A0080000B4
:1046A00002000000000000000000000033330000A2
:1046B0001142000012080000566F00006C740000E8
:1046C00073000000416E0000616C00006F67000025
:1046D000496E000032000000A00800000200000047
:1046E0000000000000000000333300001142000011
:1046F00013080000566F00006C7400007300000087
:10470000416E0000616C00006F670000496E0000A0
:1047100033000000A00800000800000000000000B6
:10472000000000000000000000000000A0090000E0
:10473000436F0000756E00007473000000450000B8
:104740006E63000030000000A008000008000000B8
:104750000000000000000000000000000000000059
:10476000A2090000436F0000756E00007473000022
:10477000004500006E63000031000000A010000042
:1047800002000000000000000000000033330000C1
:1047900011420000180A0000566F00006C740000FF
:1047A0007300000046690000656C0000645600005C
:1047B0006F6C00007461000067650000000000007D
:1047C000A010000002000000000000000000000037
:1047D00000000000000000005C0900004E6F0000B7
:1047E0006E650000005300007752000065760000FF
:1047F00069730000696F00006E000000A0100000E7
:104800000440000000000000000000000000000064
:1048100000000000000000004E6F00006E65000008
:10482000004E000056420000617500006452000016
:104830006174000065000000A0200000040000007A
:104840000000000000000000000000000000000068
:10485000780000004E6F00006E650000004E000002
:10486000565500006E690000744E0000756D000022
:104870006265000072000000A0100000044000000B
:104880000000000000000000000000000000000028
:10489000380000004E6F00006E650000004E000002
:1048A000565700006174000063680000446F000008
:1048B00067540000696D0000656F000075740000AA
:1048C00000000000A0100000020000000000000036
:1048D0000000000000000000000000009809000037
:1048E0004E6F00006E650000004500006E63000022
:1048F0004D6F00006465000030000000A010000053
:1049000002000000000000000000000000000000A5
:10491000000000009A0900004E6F00006E65000064
:10492000004500006E6300004D6F000064650000EC
:1049300031000000A0100000040000000000000092
:104940000000000000000000000000003A0000002D
:104950004E6F00006E650000004E000056450000DE
:104960006E6300004D6F00006465000030000000C1
:10497000A010000004000000000000000000000083
:1049800000000000000000003C0000004E6F00002E
:104990006E650000004E0000564500006E6300008A
:1049A0004D6F0000646500003100000070A200003F
:1049B0007EA20000DEA20000F8A2000000000000BD
:1049C00070A2000090A20000DEA20000F8A2000089
:1049D00012A3000030A300004EA300006CA300004F
:1049E0000000000070A200009EA20000DEA20000F5
:1049F000F8A2000012A3000030A300004EA30000A4
:104A00006CA30000BEA300000000000070A2000024
:104A1000BAA20000DEA20000F8A2000012A300006B
:104A200030A300004EA300006CA300008AA3000086
:104A3000A4A30000BEA300000000000070A20000BC
:104A40007EA2000090A200009EA20000BAA2000078
:104A5000DEA20000F8A2000012A3000030A30000B4
:104A60004EA300006CA300008AA30000A4A30000D2
:104A7000BEA30000E0A30000FEA300001CA40000F1
:104A80003CA4000062A400007EA400009AA40000E0
:104A9000B8A400000000000032FB07000B942000C7
:104AA0001000200049FB07008B8020004000200000
:104AB00046FB07000B802000200020004BFB070076
:104AC000E8F9370027FB07000B94200010002000B6
:104AD0003EFB07008B802000400020003BFB0700CE
:104AE0000B8020002000200040FB07000B812000ED
:104AF0001000200035FB07001B8120001000200063
:104B000032FB07002B812000100020002FFB070044
:104B10003B812000100020002CFB0700D1F937005A
:104B200010FB07000B9420001000200027FB07005B
:104B30008B8020004000200024FB07000B80200019
:104B40002000200029FB07000B812000100020001E
:104B50001EFB07001B812000100020001BFB07002C
:104B60002B8120001000200018FB07003B81200053
:104B70001000200015FB07008BA120002000200062
:104B800012FB0700B7F93700F6FA07000B94200074
:104B9000100020000DFB07008B802000400020004B
:104BA0000AFB07000B802000200020000FFB0700FD
:104BB0000B8120001000200004FB07001B81200057
:104BC0001000200001FB07002B81200010002000B6
:104BD000FEFA07003B81200010002000FBFA0700CE
:104BE0000B9A200010002000F8FA07002B9A2000F2
:104BF00010002000F5FA07008BA120002000200003
:104C0000F2FA070097F93700D6A400000502000069
:104C1000E0A4000009020000F2A400000B02000062
:104C200006A500000D0200004C25000062250000D2
:104C300090250000C42500000000000000000000D6
:104C40000000000000000000000000000000000064
:104C50000000000000000000000000000000000054
:104C60000000000000000000000000000000000044
:104C70000000000000000000000000000000000034
:104C80000000000000000000000000000000000024
:104C90000000000000000000000000000000000014
:104CA0000000000000000000000000000000000004
:104CB00000000000000000000000000000000000F4
:104CC00000000000000000000000000000000000E4
:104CD00000000000000000000000000000000000D4
:104CE00000000000000000000000000000000000C4
:104CF00000000000000000000000000000000000B4
:104D000000000000000000000000000000000000A3
:104D10000000000000000000000000000000000093
:104D20000000000000000000000000000000000083
:104D30000000000000000000000000000000000073
:104D40000000000000000000000000000000000063
:104D50000000000000000000000000000000000053
:104D60000000000000000000000000000000000043
:104D70000000000000000000000000000000000033
:104D80000000000000000000000000000000000023
:104D90000000000000000000000000000000000013
:104DA0000000000000000000000000000000000003
:104DB00000000000000000000000000000000000F3
:104DC00000000000000000000000000000000000E3
:104DD00000000000000000000000000000000000D3
:104DE00000000000000000000000000000000000C3
:104DF00000000000000000000000000000000000B3
:104E00007FEC37007EF4370022F937002BF93700AA
:104E100034F937003FF937004BF9370055F93700BF
:104E200061F937006AF9370072F9370071F9370014
:104E300070F937006FF937006EF937006DF93700F8
:104E40006CF93700C3FA3700C9FA370069F937003F
:104E500068F937009DFA370066F9370065F93700C1
:104E600064F9370063F9370062F9370061F93700F8
:104E700060F937005FF937005EF937005DF93700F8
:104E80005CF937005BF937005AF9370059F93700F8
:104E900058F9370057F9370056F9370055F93700F8
:104EA00054F9370053F9370052F9370051F93700F8
:104EB00050F937004FF937004EF937004DF93700F8
:104EC0004CF937004BF937004AF9370049F93700F8
:104ED00048F9370047F9370046F9370045F93700F8
:104EE00044F9370043F9370042F9370041F93700F8
:104EF00040F937003FF937003EF937003DF93700F8
:104F00003CF937003BF937003AF9370039F93700F7
:104F100038F9370037F9370036F9370035F93700F7
:104F200034F9370033F9370032F9370031F93700F7
:104F300030F937002FF937002EF937002DF93700F7
:104F40002CF937002BF937002AF9370029F93700F7
:104F500028F9370027F9370026F9370025F93700F7
:104F600024F9370023F9370022F9370021F93700F7
:104F700020F937001FF937001EF937001DF93700F7
:104F80001CF937001BF937001AF9370019F93700F7
:104F900018F9370017F9370016F9370015F93700F7
:104FA00014F9370013F9370012F9370011F93700F7
:104FB00010F937000FF937000EF937000DF93700F7
:104FC0000CF937000BF937000AF9370009F93700F7
:104FD00008F9370007F9370006F9370005F93700F7
:104FE00004F9370003F9370002F9370001F93700F7
:104FF00000F93700FFF83700FEF83700FDF83700FA
:1050000009000000FFFF0000010000001404000080
:105010000000000000000000000000000000000090
:105020000000000000000000000000000000000080
:105030000000000000000000000000000000000070
:105040000000000000000000000000000000000060
:105050000000000000000000000000000000000050
:105060000000000000000000000000000000000040
:1050700032000000000000000000000000000000FE
:105080000000000000800000102700001E0000004B
:10509000008000006400000000000000000000002C
:1050A0000000000000000000000000000000000000
:1050B00000000000000000000000000000000000F0
:1050C00000000000000000000000000000000000E0
:1050D00000000000000000000000000000000000D0
:1050E00000000000000000000000000000000000C0
:1050F000785600003412000000000000AA5500009D
:0200000401F009
:100000000F000000FF000000070000008300000058
:10001000C50000004000000007000000C300000011
:00000001FF
